:020000040000FA
:0600000060283D300130D4
:08000800A000030EA100831209
:1000100005191028831601178312B2308100422877
:100020008316011383120B191C28AE17280A031913
:100030002E17AE192D283B28AE13AE192A282E1FD5
:100040003B28AE1A3B28A701A601A501A801AE01D5
:10005000AE164228F030AE0542282D152E13AE12F2
:100060002708AB002608AA002508A9002808AC002C
:10007000F030AE0542282E0DA80DA50DA60DA70D3A
:10008000AE1AAE0A8B100B11210E8300A00E200EAB
:02009000090065
:1000C000203084008001840A60300402031C62280E
:1000D00034228316FF239000831283160C3085058B
:1000E000870183128501870107309900003083164C
:1000F00091009F008312C830831681008312313033
:100100009000003083168C00831210308B00BD1BD2
:100110008B28851D7D223D1BBE013D1BBF013D1F60
:10012000722281018E018F010B118B100B108C1329
:100130000C138C110C108B17AD202D19AF20082239
:10014000B30BAA28031085190314BA0DF0303A0234
:1001500003197721BD18A5229C28640008002908EE
:100160003F3C0319BB282B082A0629062C02031D35
:100170002D11031D08002D110130B7008B13203005
:10018000370783169B001C141A088312A400103032
:10019000370783169B001C141A088312A300003033
:1001A000370783169B001C141A088312A2008B17B2
:1001B00024082B02031D712923082A02031D71291B
:1001C000013003303702031D132929083F3C03196E
:1001D000FD2840302906E039031DF3283F1FF3288E
:1001E0003F13AD17012960302906E039031D0129AD
:1001F0003F1B01293F17AD170129AC1F3F13AC1B53
:100200003F1780302906F039031D0A29BF1F0A292C
:10021000BF13AD1790302906F039031D1329BF1BFA
:100220001329BF17AD17A91F7129291B712922088E
:100230002906F039A91EE039031D71292208290574
:100240000F390319472901303702031D2C293E18A5
:100250002C293E14AD174A2202303702031D3529DE
:10026000BE183529BE14AD174C2203303702031DCA
:100270003E293E193E293E15AD174E220430370265
:10028000031D4729BE194729BE15AD17522229095A
:1002900022050F390319712901303702031D552931
:1002A0003E1C55293E10AD17562202303702031D61
:1002B0005E29BE1C5E29BE10AD17582203303702DE
:1002C000031D67293E1D67293E11AD175A220430D0
:1002D0003702031D7029BE1D7029BE11AD175E22A5
:1002E0007129B70A0530370203180800BE28B60185
:1002F000B3019630B4000130B5000130B70085017C
:100300008701AD13E821AD20B30BA929031085198E
:100310000314BA0DF0303A020319D829B40BA929F5
:1003200001303702031962220230370203196622B4
:100330000330370203196A220430370203196E2290
:100340003708B6080319B6000319A729B603963073
:10035000B4002D1D83292D11A91F8329291B832951
:10036000A91E29120F30290503198329B90129185B
:10037000B90AA918B90A2919B90AA919B90AB918DB
:100380008329391983298B1320303707BC002B08A8
:10039000BB00162210303707BC002A08BB0016220B
:1003A00000303707BC002908BB0016228B17E2215A
:1003B00085018701B70AB60105303702031C83297E
:1003C00072220800043037020319080085018701F2
:1003D0001430B90033300F1E85000F1A8501FF302D
:1003E0000F1A87000F1E8701AD202D1DEA292D1140
:1003F000290A0319FF29A91FEA29291BEA290F3015
:100400002905031DE829B90BEA29850187010800A0
:10041000AD1F0800AD131030BC003E08BB00162213
:100420003030BC003F08BB00162208003C088B138C
:1004300083169B001C141A0883128B173B020319A6
:1004400008008B133B0883161C159A003C089B0080
:1004500055309D00AA309D009C1464009C182D2AE4
:100460001C1183128B170800831600309B001C148C
:100470001A088312BD00831610309B001C141A0842
:100480008312BE00831630309B001C141A0883129E
:10049000BF0008008516080005160800BD180800F2
:1004A00085140800BD18080005140800851208000E
:1004B00005120800BD18080085100800BD180800C6
:1004C000051008000508203A850008000508103AC4
:1004D000850008000508023A850008000508013A71
:1004E000850008003E188516BE180516BD180800C0
:1004F0003E198514BE1905140800B601B301B401F4
:100500003D1C852A3D10BD14882AC030BD053D1410
:100510003D083F39B60064008D2A8E2A8F2A902A22
:10052000912A3330B41B8500B41F8501B30B8B2A8D
:10053000B40B8B2A0310B60CB608031D8B2A0030AF
:10054000BC003D08BB0016220800BF1FB02A3F1B9D
:1005500085103F1B05143F1F85143F1F0510080021
:080560008510051008000800D9
:084000000500000006000200AB
:02400E00CC01E3
:1042000001008100820084008800B100B200B40087
:10421000B800A100A200FF00FF00FF00FF00FF00A8
:104220000000010001000100010001000100010087
:10423000010001000100FF00FF00FF00FF00FF0080
:10424000010000000000000000000000000000006D
:10425000000000000000FF00FF00FF00FF00FF0063
:104260000000FF00FF00FF00FF00FF00FF00FF0055
:10427000FF00FF00FF00FF00FF00FF00FF00FF0046
:10428000FF00FF00FF00FF00FF00FF00FF00FF0036
:10429000FF00FF00FF00FF00FF00FF00FF00FF0026
:1042A000FF00FF00FF00FF00FF00FF00FF00FF0016
:1042B000FF00FF00FF00FF00FF00FF00FF00FF0006
:1042C000FF00FF00FF00FF00FF00FF00FF00FF00F6
:1042D000FF00FF00FF00FF00FF00FF00FF00FF00E6
:1042E000FF00FF00FF00FF00FF00FF00FF00FF00D6
:1042F000FF00FF00FF00FF00FF00FF00FF00DD00E8
:00000001FF
